:100000000C9468050C94B0050C94B0050C94B005E4
:100010000C94B0050C94B0050C94B0050C94B0058C
:100020000C94B0050C94B0050C94B0050C94B11F61
:100030000C94901C0C94671C0C94B0050C94B005A7
:100040000C94B0050C94B0050C94B0050C94411CB4
:100050000C94B0050C94B0050C94B0050C94B0054C
:100060000C94B0050C94B0050C94B0050C94B0053C
:100070000C94B0050631FF0974A10109751500261D
:10008000FF009520750881020976150026FF00956E
:100090002075089102C005010902A1010901A10012
:1000A0008501050919012908150025019508750123
:1000B00081020501093009311581257F95027508F6
:1000C000810609381581257F950175088106050C83
:1000D0000A38021581257F950175088106C0C00583
:1000E000010980A10185021601002637001A81004E
:1000F0002AB700751095018100C0050C0901A10106
:100100008503160100269C021A01002A9C02751024
:1001100095018100C005010906A101050719E02923
:10012000E7150025019508750181020508190129C7
:100130000595057501910295017503910105071952
:100140000029F71500250195F875018102C0626F3D
:10015000756E63653A202564202564402530325849
:100160000A00646F6E652E0A00626F6F746D6167BE
:100170006963207363616E3A202E2E2E200025586D
:100180003A2530386225730A000A20203031323394
:10019000343536370A004C45443A20253032580A67
:1001A000000A4C6F6F702073746172742E0A000A1B
:1001B00055534220636F6E666967757265642E0AD7
:1001C000000A544D4B3A6133306361662F4C5546FB
:1001D000413A6436613764660A000902540003013B
:1001E00000A03209040000010301010009211101EE
:1001F00000012239000705810320000109040100E4
:100200000103010200092111010001227F000705FD
:100210008203080001090402000103000000092113
:1002200011010001222200070583032000011201B1
:10023000100100000008EDFE6464010001020001ED
:100240000E0341006C0070007300360034000000A3
:10025000080354004D004B000000040309047379A7
:100260007374656D3A20253034580A00636F6E73DD
:10027000756D65723A20253034580A003F004D3EB6
:100280002000433E20000A00257500363A2077689A
:1002900065656C5F74696D655F746F5F6D61783AF9
:1002A00020000A00257500353A20776865656C5F87
:1002B0006D61785F73706565643A20000A0025758A
:1002C00000343A2074696D655F746F5F6D61783AD0
:1002D00020000A00257500333A206D61785F737045
:1002E0006565643A20000A00257500323A20696E7F
:1002F00074657276616C286D73293A20000A0025B6
:100300007500313A2064656C6179282A31306D734B
:10031000293A20000A092D2056616C756573202D3D
:100320000A004D3E004D25643E20003F0073657479
:100330002064656661756C740A00433E20000A0003
:100340002530325820006B6579626F6172643A2003
:10035000006164645F6B65795F6269743A20636110
:100360006E2774206164643A20253032580A006494
:10037000656C5F6B65795F6269743A2063616E27B3
:10038000742064656C3A20253032580A007E10369D
:100390000E0F12272D7F37383334132F2E7C7D29F3
:1003A000283130742A787939042B14351E7B641D6A
:1003B000161A081F207A1B0709151721222C061967
:1003C0000A1C1823246505110B0D0C2526290A008B
:1003D0002575002F002575005D280025640020008C
:1003E000256400200025640020002564007C002591
:1003F000303258006D6F7573656B6579205B627480
:100400006E7C782079207620685D287265702F6177
:10041000636C293A205B006D6F7573653A205B252C
:100420003032587C25642025642025642025645DB5
:100430000A000A002530325820000A253034583A84
:100440002000656570726F6D3A000A002575002EF8
:100450006E6B726F3A20000A002575002E7377616B
:10046000705F6261636B736C6173685F6261636B21
:1004700073706163653A20000A002575002E73775A
:1004800061705F67726176655F6573633A20000A29
:10049000002575002E6E6F5F6775693A20000A00AF
:1004A0002575002E737761705F72616C745F72677F
:1004B00075693A20000A002575002E737761705F18
:1004C0006C616C745F6C6775693A20000A00257571
:1004D000002E636170736C6F636B5F746F5F636F2B
:1004E0006E74726F6C3A20000A002575002E7377C7
:1004F00061705F636F6E74726F6C5F636170736C59
:100500006F636B3A20000A0025303258006B657922
:100510006D61705F636F6E6669672E7261773A20F6
:10052000000A002575002E6D6F7573653A20000A6C
:10053000002575002E6B6579626F6172643A200048
:100540000A002575002E6D61747269783A20000AE0
:10055000002575002E656E61626C653A20000A0008
:10056000253032580064656275675F636F6E666937
:10057000672E7261773A20000A002575006465666F
:1005800061756C745F6C617965723A20000A092D9F
:10059000204D61676963202D0A643A0964656275BC
:1005A000670A783A096465627567206D61747269DB
:1005B000780A6B3A096465627567206B6579626FCA
:1005C0006172640A6D3A096465627567206D6F75C2
:1005D00073650A763A0976657273696F6E0A733AC3
:1005E000097374617475730A633A09636F6E736F8C
:1005F0006C65206D6F64650A302D343A096C617941
:100600006572302D34284631302D4634290A506128
:1006100075733A09626F6F746C6F616465720A6515
:100620003A09656570726F6D0A6E3A094E4B524F0A
:100630000A000A092D20436F6E736F6C65202D0A26
:100640004553432F713A09717569740A6D3A096D02
:100650006F7573656B65790A003F004E4B524F3AD8
:10066000206F66660A004E4B524F3A206F6E0A00AA
:1006700074696D65725F72656164333228293A204E
:100680002530346C580A006B6579626F6172645F63
:100690006E6B726F3A2025580A006B6579626F6144
:1006A00072645F69646C653A2025580A006B65794D
:1006B000626F6172645F70726F746F636F6C3A2007
:1006C00025580A00686F73745F6B6579626F617299
:1006D000645F6C65647328293A2025580A000A096A
:1006E0002D20537461747573202D0A004743433ADB
:1006F00020372E332E30204156522D4C4942433A5A
:1007000020322E302E30204156525F415243483A1B
:100710002061767233350A004F5054494F4E533A98
:10072000204C55464120424F4F544D4147494320AC
:100730004D4F5553454B45592045585452414B4513
:100740005920434F4E534F4C4520434F4D4D414E42
:1007500044204E4B524F204B45594D41505F53451D
:100760004354494F4E20343039360A004255494CE3
:10077000443A20613330636166202830323A33379F
:100780003A3539204E6F76203237203230323329D5
:100790000A005649443A2030784645454428544D8D
:1007A0004B29205049443A20307836343634284199
:1007B0006C7073363429205645523A2030783030E8
:1007C00030310A00444553433A20544D4B206B6569
:1007D00079626F617264206669726D7761726520FB
:1007E000666F7220416C707336340A000A092D203E
:1007F00056657273696F6E202D0A000A6D6F7573EE
:10080000653A206F66660A000A6D6F7573653A2057
:100810006F6E0A000A6B6579626F6172643A206FCD
:1008200066660A000A6B6579626F6172643A206FCE
:100830006E0A000A6D61747269783A206F66660A02
:10084000000A6D61747269783A206F6E0A000A645A
:10085000656275673A206F6E0A000A6465627567A3
:100860003A206F66660A000A0A626F6F746C6F61E5
:100870006465722E2E2E2000433E20006565636F56
:100880006E6669673A0A006D6B5F776865656C5FD5
:1008900074696D655F746F5F6D6178203D202564BC
:1008A0000A006D6B5F776865656C5F6D61785F737B
:1008B00070656564203D2025640A006D6B5F746976
:1008C0006D655F746F5F6D6178203D2025640A005F
:1008D0006D6B5F6D61785F7370656564203D202589
:1008E000640A006D6B5F696E74657276616C203DA1
:1008F0002025640A006D6B5F64656C6179203D2082
:1009000025640A006D6B5F776865656C5F74696D5F
:10091000655F746F5F6D6178203D2025640A006D0E
:100920006B5F776865656C5F6D61785F7370656537
:1009300064203D2025640A006D6B5F74696D655FFE
:10094000746F5F6D6178203D2025640A006D6B5FD8
:100950006D61785F7370656564203D2025640A00D1
:100960006D6B5F696E74657276616C203D202564E5
:100970000A006D6B5F64656C6179203D2025640A17
:100980000077686572652064656C74613A206375F0
:1009900072736F723D25642C20776865656C3D2508
:1009A000640A53656520687474703A2F2F656E2E43
:1009B00077696B6970656469612E6F72672F7769FB
:1009C0006B692F4D6F7573655F6B6579730A000AEC
:1009D000092D204D6F7573656B6579202D0A455380
:1009E000432F713A09717569740A313A0964656C6B
:1009F0006179282A31306D73290A323A09696E7497
:100A0000657276616C286D73290A333A096D6178D5
:100A10005F73706565640A343A0974696D655F7463
:100A20006F5F6D61780A353A09776865656C5F6D4F
:100A300061785F73706565640A363A097768656541
:100A40006C5F74696D655F746F5F6D61780A0A70C1
:100A50003A097072696E742076616C7565730A6408
:100A60003A097365742064656661756C74730A7500
:100A7000703A092B310A646F776E3A092D310A708A
:100A80006775703A092B31300A7067646F776E3A78
:100A9000092D31300A0A7370656564203D20646554
:100AA0006C7461202A206D61785F737065656420C5
:100AB0002A2028726570656174202F2074696D6525
:100AC0005F746F5F6D6178290A004C25640A00002D
:100AD00011241FBECFEFD4E0DEBFCDBF04B603FEAE
:100AE00028C08091C0029091C102A091C202B09131
:100AF000C3028730904BA740B04BD9F41092C0028C
:100B00001092C1021092C2021092C30214BE0FB61C
:100B1000F894A8958091600088618093600010929D
:100B200060000FBE1092010810920008E0E0F8E3A8
:100B3000099511E0A0E0B1E0EEEDFCE402C0059003
:100B40000D92A433B107D9F722E0A4E3B1E001C0CC
:100B50001D92A03CB207E1F70E947F200C946D2605
:100B60000C940000FF93EF93E0913401F091350174
:100B7000309709F00995EF91FF910895FC01859157
:100B8000803011F0EFDFFBCF0895FF27E0E230E285
:100B900047FF0CC0419597FF09C0EDE26095709545
:100BA00080959095611D711D811D911D27FF02C0CB
:100BB000219530E350E2AA27660F771F881F991FFF
:100BC000AA1FA41710F0A41B63955A95A9F7AA3081
:100BD00008F0A95FA05DAF93F395611571058105DC
:100BE000910541F7ED3211F4EF93F395F21718F4F4
:100BF0003F93F395FBCF8F91B5DFFA95E1F7089519
:100C0000E991F9918591803021F0853219F0AADFC0
:100C1000F9CF089520E0E89455915532C1F350334F
:100C200011F4689455915A3348F4505390F3220FBD
:100C3000022E220F220F200D250FF4CF0EF4219546
:100C400089919991533619F3533729F1533559F155
:100C5000BC0188279927E8945C3621F48991999101
:100C600068945591543639F446EF7EF077FF0DC005
:100C70008FEF9FEF0AC055374AE039F0583540E111
:100C800021F0523642E009F00895FF93EF937DDFA3
:100C9000EF91FF91B7CFFF93EF93FC0181918030EB
:100CA000B9F360DFFBCFFF93EF9368DFF1CFDF9302
:100CB000CF93CDB7DEB72596A3DFCF91DF9108950F
:100CC000803FC1F48091B20287FD1092B202809100
:100CD000B10281110EC08091B20281110AC08091CF
:100CE000B302811106C08091B402811102C010923A
:100CF000AB020895813F29F48091B20218162CF3BB
:100D0000E6CF9091B102823F29F497FFE0CF109295
:100D1000B102DDCF833F19F41916CCF3D8CF893F48
:100D200039F48091B302181694F61092B302CFCF23
:100D30008A3F29F48091B30287FFC9CFF6CF8B3F5A
:100D400039F48091B40287FFC2CF1092B402BFCFB2
:100D50008C3F29F48091B4021816BCF3B8CF843FBD
:100D600031F48091B0028E7F8093B002B0CF853F86
:100D700021F48091B0028D7FF7CF863F21F48091DE
:100D8000B0028B7FF1CF873F21F48091B002877F43
:100D9000EBCF883F21F48091B0028F7EE5CF8D3F6D
:100DA00031F48091AA028E7F8093AA0290CF8E3F69
:100DB00021F48091AA028D7FF7CF8F3F09F087CF72
:100DC0008091AA028B7FF0CF8091AA0280FF0CC095
:100DD0006091140170E0759567957595679561153B
:100DE000710559F1862F089581FF06C060911401A5
:100DF00070E075956795F3CF6091140170E082FD06
:100E00000CC06091AB026623A9F020911301809180
:100E1000140190E0621730F0BC0160387105F8F2FF
:100E20008FE7089570E00E942E26622F70E00E94E6
:100E30003F26F3CF61E070E0D5CF81E00895809147
:100E4000AA0280FF11C08091160190E065E070E079
:100E50000E942E26959587959595879580389105C2
:100E6000B0F50097B1F1089581FF0AC08091160195
:100E700090E065E070E00E942E2695958795EECF74
:100E800082FF08C08091160190E065E070E00E944A
:100E90002E26E4CF3091AB023323B1F0209115011F
:100EA0008091160190E065E070E00E942E26BC0162
:100EB0003217A0F6832F90E00E942E26622F70E05A
:100EC0000E943F26CB01CACF85E090E008958FE7CE
:100ED000089581E00895803F31F40E941F078195B5
:100EE0008093B2020895813F19F40E941F07F8CF42
:100EF000823F31F40E941F0781958093B1020895CB
:100F0000833F19F40E941F07F8CF893F29F40E94FC
:100F1000E4068093B30208958A3F21F40E94E40618
:100F20008195F7CF8B3F31F40E94E4068195809341
:100F3000B40208958C3F19F40E94E406F8CF843F70
:100F400031F48091B00281608093B0020895853FB2
:100F500021F48091B0028260F7CF863F21F4809126
:100F6000B0028460F1CF873F21F48091B0028860A5
:100F7000EBCF883F21F48091B0028061E5CF8D3FB7
:100F800031F48091AA0281608093AA0208958E3F75
:100F900021F48091AA028260F7CF8F3FB9F7809148
:100FA000AA028460F1CFE72FF0E093E0EE0FFF1F7D
:100FB0009A95E1F7E60FF11DE357FC4F6491E62F98
:100FC000E295E77090E023E0880F991F2A95E1F7FA
:100FD0008E0F911D34E0880F991F3A95E1F7E62FA7
:100FE000EF70E80FF92FF11DEE0FFF1FE050F849E9
:100FF000859194910895AF92BF92CF92DF92EF9234
:10100000FF921F93CF93DF935C0182EAC82E82E0A8
:10101000D82E10E0F601E1906F01D0E0C0E0F12C95
:10102000C7010C2E02C0959587950A94E2F780FFC0
:101030001DC06C2F712F80E00E94D3078A159B057D
:1010400051F0292F207E392F307C11F0203A71F495
:101050008A151B0459F481E0DF91CF911F91FF9015
:10106000EF90DF90CF90BF90AF9008952196C83059
:10107000D105B1F61F5F183069F680E0EDCFCF9350
:10108000DF93EC018CE290E00E94FB07882329F0BB
:10109000CE01DF91CF910C94FB0780E0DF91CF91DF
:1010A00008952FB7F8948091B5029091B602A0915F
:1010B000B702B091B8022FBF08958238F1F080F4E2
:1010C000813309F44DC038F4893209F444C08A32BE
:1010D00009F44BC008958533C9F1893371F008953F
:1010E000833EF9F028F4803E71F0823E91F008953D
:1010F000863EF1F0873E21F1089590915902937058
:10110000B1F080EE08959091590290FF10C089E3EC
:1011100008959091590292FF0AC094FF2BC080E07D
:1011200008959091590292FD27C094FDF8CF08953B
:101130009091590293FFFBCF94FDF1CF87EE089574
:101140009091590293FFF1CF86EE08959091590244
:1011500095FD14C008959091590295FD11C0089510
:101160009091590296FD0EC008959091590296FDF6
:101170000BC0089583EE089582EE089589E20895E4
:1011800085E308958AE2089581E3D1CF4F925F927B
:101190006F927F929F92AF92BF92CF92DF92EF9227
:1011A000FF920F931F93CF93DF9300D000D01F9235
:1011B000CDB7DEB76B837C838D837A018C819D8173
:1011C000892B49F08FEFF81204C081E09FEF491797
:1011D00019F080E001C081E080FF17C080E090E05E
:1011E0000F900F900F900F900F90DF91CF911F9164
:1011F0000F91FF90EF90DF90CF90BF90AF909F90B6
:101200007F906F905F904F9008950F2D10E0CE2C3F
:10121000D12C8B81882309F44FC040905A02509002
:101220005B0260905C0270905D028091BC029091C4
:10123000BD02A091BE02B091BF02482A592A6A2A73
:101240007B2A2FE1A22EB12C9A2CD301C2010A2CA9
:1012500004C0B695A795979587950A94D2F780FD17
:1012600024C081E0A81AB10878F7912CF80193E026
:10127000EE0FFF1F9A95E1F7E25AFD4FEC0DFD1DB1
:101280009082B701892D0E94D307192F982F212F03
:1012900022952F70243018F02A50223018F40E9422
:1012A0005D08982F892F912F9BCFB7018A2D0E941F
:1012B000D3070197B1F2DACFF80183E0EE0FFF1FF9
:1012C0008A95E1F7E25AFD4FEC0DFD1D9080D9CFD4
:1012D00041E050E060E070E004C0440F551F661F1D
:1012E000771F8A95D2F740955095609570958091BB
:1012F0005A0290915B02A0915C02B0915D0284233E
:101300009523A623B72380935A0290935B02A09360
:101310005C02B0935D02089541E050E060E070E04F
:1013200004C0440F551F661F771F8A95D2F780911E
:101330005A0290915B02A0915C02B0915D02842BF5
:10134000952BA62BB72B80935A0290935B02A09308
:101350005C02B0935D02089580915802909127023B
:10136000981301C008958F5F8770FACF1F93CF93B2
:10137000DF9300D000D01F92CDB7DEB7942F498302
:10138000252F5A836B837C838D834C815D8181E023
:10139000452B31F02F3F19F481E09F3F09F080E0A9
:1013A000182F117080FD2CC049815A816B817C817E
:1013B0008D810E94C608292F22952F702C3078F439
:1013C0002A30A8F422502230C8F0812F0F900F90BD
:1013D0000F900F900F90DF91CF911F9108952C30B7
:1013E00011F02F3091F793FB112710F9EECF803CCD
:1013F00028F0803E50F3815F833038F311E0E5CF71
:1014000010E0E3CFE091AC02F091AD02309721F013
:101410000190F081E02D099480E008951092E2009F
:101420001092E100E0EEF0E0808181608083E8EDE1
:10143000F0E080818F77808319BCE3E6F0E0808163
:10144000816080831092ED0108950E940E0AF89445
:1014500087E797E7909301088093000887E090EB77
:10146000DC018093C0029093C102A093C202B093AA
:10147000C30288E19CE00FB6F894A89580936000C1
:101480000FBE90936000FFCFFC0180911A029091F3
:101490001B0286179707A0F06115710529F490913A
:1014A000E8009E779093E80090E06115710551F493
:1014B000911108C08091E80082FF32C080E0089559
:1014C000BC01F2CF809112028823B1F18530B1F1D5
:1014D0008091E80083FD2EC08091E80082FDEACF74
:1014E0008091E80080FFE1CF2091F20030E06115AB
:1014F000710519F02830310558F091E02830310598
:1015000009F090E02091E8002E772093E800CDCFFD
:1015100081918093F100615071092F5F3F4FE7CFB8
:1015200080911202882341F0853041F08091E800DB
:1015300083FFC0CF81E0089582E0089583E008959D
:101540002091E4003091E50085E69091EC0090FF59
:1015500006C09091E80090FF06C080E00895909149
:10156000E80092FDFACF90911202992391F0953004
:1015700091F09091EB0095FD10C04091E4005091E6
:10158000E5002417350709F381509A01F1F684E04C
:10159000089582E0089583E0089581E00895EF9230
:1015A000FF920F931F93CF937C018B010E94A00A9F
:1015B000C82F811117C08091E80085FD0BC0809174
:1015C000E8008E778093E8000E94A00A882399F3B0
:1015D000C82F08C0F70181917F018093F10001506D
:1015E000110949F78C2FCF911F910F91FF90EF9028
:1015F00008958091140287FF13C08091E80082FF54
:1016000006C08091E8008B778093E80004C0809149
:1016100012028111F2CF0895809112028823D9F32A
:101620008091E80080FFF8CF8091E8008E77ECCFC2
:10163000982F9093E900242F762F50E0891731F0EE
:101640007091EC002091ED005091F00021FD07C059
:101650009F5F953071F78093E90081E008953091A4
:10166000EB003E7F3093EB003091ED003D7F3093F7
:10167000ED003091EB0031603093EB007093EC00A3
:101680002093ED005093F0002091EE0027FDE0CF75
:1016900080E008958091EF0108958091D901811132
:1016A00013C09FB7F8944091B5025091B602609173
:1016B000B7027091B8029FBF443C59406105710563
:1016C00018F081E08093D9010895EF92FF920F9373
:1016D0001F93CF93DF93D82F0FB607FE46C080919C
:1016E0001202843079F08091030190E001962091FC
:1016F000050130E082239323209104012817190665
:1017000009F0C9C00E944D0B81110FC080910301E7
:1017100090E001962091050130E0822393232091EF
:1017200004012817190609F0B6C00E9451088C015F
:10173000C091E900CF708091EC0080FD37C080E05F
:10174000C82B83E08093E90085E0E82E8091EB00D0
:1017500085FD08C08091EB0080FF04C08091EE0001
:1017600087FD44C0CF70C093E900E09103018E2F44
:1017700090E001962091050130E08223932320918F
:1017800004012817190609F47EC080910101909187
:101790000201E80FF92FF11DD083809103018F5FC3
:1017A000909105018923809303016DC080E8C8CF23
:1017B000E0910101F0910201E80FF11D90818F5F2E
:1017C000209105018223809304019093F100809180
:1017D000E80085FD0BC08091E80080FF07C0809184
:1017E000E8008E778093E800E09200018091040188
:1017F00090910301981741F19091E80095FDD8CFA1
:1018000080E029C01092F1002EC08091030190E089
:1018100001962091050130E0822393232091040159
:101820002817190609F09ECFF0900001FF2009F457
:1018300099CF0E9451088017910709F487CFFA9435
:10184000F09200018C0182CF8091E80085FFD8CF13
:10185000D093F10081E09091F200992379F090917A
:10186000E80090FF0BC09091E80095FDCBCF9091E0
:10187000E8009E779093E800E0920001882329F227
:10188000CF70C093E90080E0DF91CF911F910F915D
:10189000FF90EF900895E091030177CF8AB18078AF
:1018A0008AB98BB180788BB93A9842980895833081
:1018B000C9F128F4813061F0823019F10895853042
:1018C00009F452C008F43FC0863009F45EC00895A0
:1018D00080911801681790F4861B809318018091FD
:1018E00018011F928F9382E799E09F938F930E9434
:1018F00057060F900F900F900F90089510921801B7
:10190000EECF80911701681750F4861B8093170162
:10191000809117011F928F9380E699E0E6CF109295
:101920001701F6CF80911601681750F4861B80933B
:101930001601809116011F928F938DE499E0D5CF07
:1019400010921601F6CF80911501681750F4861B8E
:1019500080931501809115011F928F9388E399E080
:10196000C4CF10921501F6CF80911401681750F47E
:10197000861B80931401809114011F928F938FE135
:1019800099E0B3CF10921401F6CF8091130168173C
:1019900050F4861B80931301809113011F928F9343
:1019A00084E099E0A2CF10921301F6CF833009F4BE
:1019B00045C028F4813061F0823049F108958530C6
:1019C00009F46AC008F451C0863009F47CC0089557
:1019D00080911801482F460F5527551F4F3F51053D
:1019E00094F4680F60931801809118011F928F93EF
:1019F00085EF98E09F938F930E9457060F900F906A
:101A00000F900F9008958FEF80931801EDCF809184
:101A10001701482F460F5527551F4F3F510554F4C6
:101A2000680F60931701809117011F928F9383EEC7
:101A300098E0E0CF8FEF80931701F5CF80911601EA
:101A4000482F460F5527551F4F3F510554F4680F37
:101A500060931601809116011F928F9380ED98E09C
:101A6000C9CF8FEF80931601F5CF80911501482FD4
:101A7000460F5527551F4F3F510554F4680F60938B
:101A80001501809115011F928F938BEB98E0B2CFD7
:101A90008FEF80931501F5CF80911401482F460FE9
:101AA0005527551F4F3F510554F4680F609314019B
:101AB000809114011F928F9382EA98E09BCF8FEF61
:101AC00080931401F5CF80911301482F460F5527BD
:101AD000551F4F3F510554F4680F609313018091D7
:101AE00013011F928F9387E898E084CF8FEF809344
:101AF0001301F5CF90911201992369F19091110191
:101B0000992349F1E82FE695E695E695EF3191F0B6
:101B1000F0E0EA54FE4F877021E030E0A90102C0F6
:101B2000440F551F8A95E2F7CA0180959181892358
:101B3000818308959091BB0290FF19C01F928F93EB
:101B40008FE693E09F938F930E9457060F900F901C
:101B50000F900F900895E6EBF1E024ED31E09281D3
:101B6000891301C0128231962E173F07C1F70895DD
:101B700090911201992349F190911101992329F132
:101B8000E82FE695E695E695EF3171F0F0E0EA543E
:101B9000FE4F877021E030E001C0220F8A95EAF7FE
:101BA0008181822B818308959091BB0290FF1EC09A
:101BB0001F928F9381E593E09F938F930E94570626
:101BC0000F900F900F900F900895A8EBB1E0EFEFFA
:101BD00090E02D91821751F0EF3F19F4211101C0CF
:101BE000E92F9F5F9E31A9F7EF3F09F408950E2E6C
:101BF000000CFF0BEA54FE4F82830895CF93DF93CE
:101C000020911E0230911F022817390701F190938D
:101C10001F0280931E02E091AC02F091AD0230975A
:101C2000B1F0EC010084F185E02D09958091BB02B3
:101C30008570853061F4DF93CF938CE692E09F93BB
:101C40008F930E9457060F900F900F900F90DF9187
:101C5000CF910895CF93DF9320911C0230911D0204
:101C60002817390701F190931D0280931C02E0911F
:101C7000AC02F091AD023097B1F0EC010680F78133
:101C8000E02D09958091BB028570853061F4DF936A
:101C9000CF938EE592E09F938F930E9457060F900B
:101CA0000F900F900F90DF91CF9108958FEC99E0F6
:101CB0000E94BE051F9281E08F931F9285E08F9353
:101CC00081E899E09F938F930E9457060F900F90A1
:101CD0000F900F900F900F900895CF938091BB02BB
:101CE00083FF7EC084EF93E00E94BE058091B00226
:101CF0001F928F938FEE93E09F938F930E945706CE
:101D00008DEE93E00E94BE058091B102282F082E2F
:101D1000000C330B3F938F938AEE93E09F938F9346
:101D20000E94570688EE93E00E94BE058091B202A1
:101D3000282F082E000C330B3F938F9385EE93E0F2
:101D40009F938F930E94570683EE93E00E94BE05F7
:101D50008091B302282F082E000C330B3F938F93F2
:101D600080EE93E09F938F930E9457068EED93E051
:101D70000E94BE058091B402282F082E000C330B60
:101D80003F938F938BED93E09F938F930E94570621
:101D900088ED93E00E94BE058091AB021F928F9365
:101DA00085ED93E09F938F930E94570683ED93E018
:101DB0000E94BE058091AA021F928F9380ED93E04E
:101DC0009F938F930E9457068DEC93E00E94BE056F
:101DD0008DB79EB74C960FB6F8949EBF0FBE8DBFC1
:101DE000E091AC02F091AD023097F1F1C091B002F8
:101DF0000480F581E02D80EB92E00995C093B0025C
:101E00008091BB0283FF30C08091B402282F082E3E
:101E1000000C330B3F938F938091B302282F082E31
:101E2000000C330B3F938F938091B202282F082E22
:101E3000000C330B3F938F938091B102282F082E13
:101E4000000C330B3F938F931F92CF9387E194E065
:101E50009F938F930E9457068DB79EB70C960FB62F
:101E6000F8949EBF0FBE8DBF0E9451089093AF02A1
:101E70008093AE02CF9108950F931F93CF93DF937A
:101E80008091A00290919F02892B8093B60190913E
:101E90009E02992389F0892B8093B601E7EBF1E04C
:101EA00026ED31E080E0919191118F5F2E173F0771
:101EB000D1F7811110929E02E091AC02F091AD0237
:101EC0003097B1F10280F381E02D86EB91E0099526
:101ED0008091BB0282FF2CC080FF04C086E493E0A7
:101EE0000E94BE05D0E0C0E000E413E08091BB0298
:101EF00080FF0EC0FE01EA54FE4F80811F928F9337
:101F00001F930F930E9457060F900F900F900F9002
:101F10002196C032D10551F78091BB0280FF08C0E5
:101F20008EE393E0DF91CF911F910F910C94BE054A
:101F3000DF91CF911F910F9108951092A0021092FE
:101F40009F02E7EBF1E0119281E0E63DF807D9F757
:101F50000E943C0F85E0E0EBF2E0DF011D928A95E4
:101F6000E9F71092AB021092AA020E946D0E90E067
:101F700080E00E942A0E90E080E00C94FE0DCF934A
:101F8000C82F1F928F938AEC9AE09F938F930E94A1
:101F9000570681E090E0A0E0B0E004C0880F991FF0
:101FA000AA1FBB1FCA95D2F78093BC029093BD02B3
:101FB000A093BE02B093BF020F900F900F900F90AE
:101FC000CF910C949D0F882341F080959091A002B1
:101FD00089238093A0020C943C0F0895882339F044
:101FE0009091A002892B8093A0020C943C0F08953D
:101FF000CF93DF93882309F45DC09EE7980F933059
:1020000020F5C2E0D9E3823831F0C4E0D7E4833868
:1020100011F4C1E0D3E50E94020A8C2309F44AC0FE
:102020008D2F0E94B80D0E943C0F2FEF41EE54E01F
:10203000215040405040E1F700C000008D2F0E9429
:102040007A0DDF91CF910C943C0F9CEF980F913A51
:10205000B0F390E2980F983088F4877021E030E078
:10206000A90102C0440F551F8A95E2F7CA01809565
:102070009091A00289238093A002E3CF9BE5980F63
:10208000933030F490E080E0DF91CF910C942A0EF1
:1020900098E5980F973130F490E080E0DF91CF9190
:1020A0000C94FE0D803F30F00E946006DF91CF91CE
:1020B0000C946D0EDF91CF910895CF93DF9300D0F4
:1020C0001F92CDB7DEB720911202243041F5209146
:1020D0001001222321F123E029839B838A8382E05C
:1020E0008093E9008FEF9091E800815095FD06C044
:1020F00095ED9A95F1F700008111F5CF8091E800F8
:1021000085FF0DC050E040E063E070E0CE01019635
:102110000E94CF0A8091E8008E778093E8000F90AC
:102120000F900F90DF91CF910895CF93DF9300D060
:102130001F92CDB7DEB720911202243081F5209195
:102140001001222361F119821A821B8222E0298365
:102150008138910520F0805891099B838A8382E021
:102160008093E9008FEF9091E800815095FD06C0C3
:1021700095ED9A95F1F700008111F5CF8091E80077
:1021800085FF0DC050E040E063E070E0CE010196B5
:102190000E94CF0A8091E8008E778093E8000F902C
:1021A0000F900F90DF91CF9108952091120224306B
:1021B00049F522E02093E9002FEF3091E80021500B
:1021C00035FD06C035ED3A95F1F700002111F5CF48
:1021D0002091E80025FF16C02091100150E040E05A
:1021E00063E070E0222339F021E02093F10050E019
:1021F00040E065E070E00E94CF0A8091E8008E77B1
:102200008093E8000895CF93DF9320911202243049
:10221000D9F4EC01809112018823F1F08091110131
:102220008823D1F081E08093E90081E8815021F09A
:102230009091E80095FF0BC08091E80050E040E0ED
:1022400060E270E085FD1AC0DF91CF9108959AE2B7
:102250009A95F1F700C0EACF81E08093E90081E828
:10226000815021F09091E80095FF19C08091E8001D
:1022700085FFEACF50E040E068E070E0CE010E94C8
:10228000CF0A8091E8008E778093E80080E2FE011B
:10229000A0EFB1E001900D928A95E1F7D5CFEFE381
:1022A000F1E03197F1F700C00000DACFAF92BF92B2
:1022B000CF92DF92EF92FF920F931F93CF93DF9312
:1022C0000AED11E07801D0E0C0E0AA24A3948EE4E6
:1022D000C82E81E0D82EEC2FE150E73060F4F0E01A
:1022E000EC58FE4E0C945326F411F711FA11FD111F
:1022F000001203120612509A589820EA2A95F1F714
:10230000B3B0B094D7012D917D012B15B9F1809117
:10231000D801882341F18091BB0280FF24C0409105
:10232000D6015091D7013FB7F8948091B5029091B2
:10233000B602A091B702B091B8023FBF2B251F9201
:102340002F93DF93CF93841B950B9F938F93DF92F3
:10235000CF920E9457068DB79EB708960FB6F89495
:102360009EBF0FBE8DBFF7013197B082A092D801FA
:102370000E9451089093D7018093D6010E944E0C81
:102380002196C830D10509F0A6CF8091D8018823C5
:10239000F9F02091D6013091D7014FB7F894809190
:1023A000B5029091B602A091B702B091B8024FBFAA
:1023B000821B930B059760F0E2EAF2E0D8018D9161
:1023C0008D018193B1E0023E1B07C1F71092D80145
:1023D00081E0DF91CF911F910F91FF90EF90DF90FF
:1023E000CF90BF90AF900895519A599886CF529A46
:1023F0005A9883CF539A5B9880CF549A5C987DCF3C
:10240000559A5D987ACF569A5E9877CF3A9A4298C5
:1024100074CFEF92FF920F931F93CF93DF938B3183
:1024200009F40FC208F04AC08E3009F41AC2B8F499
:10243000873009F4EFC148F4863009F4D9C189E541
:1024400096E00E94BE05C0E077C2883009F467C0FC
:102450008B30A9F78DE895E00E94BE05C7C1813198
:1024600009F45CC278F4803151F79091BB02892F56
:10247000877F93FF88608093BB0283FF02C288E05E
:1024800098E0D9C1863109F4FFC18931C1F68CEEDB
:1024900097E00E94BE0584EC97E00E94BE0582E9A9
:1024A00097E00E94BE058CE697E00E94BE0588E199
:1024B00097E00E94BE058CEE96E0CECF853361F0AA
:1024C00078F4873249F028F48E3108F4B8CF8D5172
:1024D00004C0893209F0B3CF80E00E94BF0F86C1EB
:1024E000833438F48A3308F032C2883309F4B2CF27
:1024F000A6CF833489F3883409F0A1CF0E949D0FC1
:1025000087E698E00E94BE059FEF23ED80E391509F
:1025100020408040E1F700C000000E94250A8CE7BF
:1025200098E00E94BE058DE795E00E94BE0583E01D
:1025300090E00E94C4241F928F938AE795E09F93B6
:102540008F930E94570688E795E00E94BE0582E0BF
:1025500090E00E94C424C82F85E695E00E94BE0545
:102560001F92CF9380E695E09F938F930E9457062A
:102570008EE595E00E94BE0584E595E00E94BE05CB
:102580008C2F81701F928F9381E595E09F938F939D
:102590000E9457068FE495E00E94BE0585E495E011
:1025A0000E94BE05C1FB882780F91F928F9382E4A9
:1025B00095E09F938F930E94570680E495E00E94D8
:1025C000BE0584E395E00E94BE05C2FB882780F922
:1025D0001F928F9381E395E09F938F930E945706FC
:1025E0008FE295E00E94BE0586E295E00E94BE055E
:1025F000C3FBCC27C0F91F92CF9383E295E09F9352
:102600008F930E94570681E295E00E94BE0584E008
:1026100090E00E94C424C82F8DE095E00E94BE0582
:102620001F92CF9388E095E09F938F930E94570667
:1026300086E095E00E94BE058DEE94E00E94BE0506
:102640008C2F81701F928F938AEE94E09F938F93CB
:102650000E9457068DB79EB780960FB6F8949EBF1E
:102660000FBE8DBF88EE94E00E94BE0581ED94E020
:102670000E94BE05C1FB882780F91F928F938EECC4
:1026800094E09F938F930E9457068CEC94E00E94F5
:10269000BE058AEB94E00E94BE05C2FB882780F944
:1026A0001F928F9387EB94E09F938F930E9457061E
:1026B00085EB94E00E94BE0583EA94E00E94BE058B
:1026C000C3FB882780F91F928F9380EA94E09F9341
:1026D0008F930E9457068EE994E00E94BE0584E91C
:1026E00094E00E94BE05C4FB882780F91F928F9357
:1026F00081E994E09F938F930E9457068FE894E0BE
:102700000E94BE058DE794E00E94BE05C5FB8827A8
:1027100080F91F928F938AE794E09F938F930E9492
:10272000570688E794E00E94BE058CE594E00E947D
:10273000BE05C6FB882780F91F928F9389E594E038
:102740009F938F930E94570687E594E00E94BE05F1
:102750008FE494E00E94BE05C7FBCC27C0F91F920E
:10276000CF938CE494E09F938F930E9457068AE462
:1027700094E00E94BE0582E494E09F938F930E94B0
:1027800057068DB79EB74E960FB6F8949EBF0FBEF4
:102790008DBFD0E0C0E08AE3E82E84E0F82E04E3A9
:1027A00014E0209751F41F921F92FF92EF920E9423
:1027B00057060F900F900F900F90CE010E94C424E7
:1027C0001F928F931F930F930E94570621960F908D
:1027D0000F900F900F90C031D10519F782E394E06C
:1027E0009F938F930E9457060F900F90C1E0A4C053
:1027F0008091BB02817F8E7F8093BB0282E396E053
:102800000E94BE0588E798E00E94BE0581E08093A3
:10281000BA02ECCF8091BB0280FF0BC08AE598E042
:102820000E94BE058091BB02817F8E7F8093BB0298
:10283000DDCF8EE498E00E94BE058091BB028160EE
:10284000F5CF9091BB02892F8D7F91FF826080939D
:10285000BB0281FF03C081E498E0EDCF83E398E001
:10286000FBCD9091BB02892F8B7F92FF8460809378
:10287000BB0282FF03C084E298E0DDCF84E198E0F0
:10288000EBCD8BEF97E0E8CD8EED96E00E94BE0594
:102890000E94020A1F928F9384EC96E09F938F937D
:1028A0000E945706809112011F928F938DEA96E045
:1028B0009F938F930E9457068091B9021F928F9326
:1028C0008AE996E09F938F930E94570680911101A9
:1028D0001F928F9387E896E09F938F930E945706ED
:1028E0002FB7F8948091B5029091B602A091B702EB
:1028F000B091B8022FBFBF93AF939F938F9380E7A0
:1029000096E09F938F930E9457068DB79EB7469689
:102910000FB6F8949EBF0FBE8DBF68CF0E949D0F6B
:10292000C091110181E0C827C0931101CC2361F04F
:1029300086E696E00E94BE058C2FDF91CF911F9115
:102940000F91FF90EF9008958BE596E085CD895328
:10295000C4CDCF93DF93882309F4BDC0C82F8EE781
:102960008C0F833030F5C238F1F0C338F9F0C4E091
:10297000D7E40E94020A8C2309F0ADC08D2F0E947B
:10298000B80D0E943C0F2FEF81EE94E02150804063
:102990009040E1F700C000008D2F0E947A0DDF917A
:1029A000CF910C943C0FC2E0D9E3E3CFC1E0D3E573
:1029B000E0CF8CEF8C0F813A08F03AC18091BA02D7
:1029C000813099F040F08230E9F11092BA028C2FF8
:1029D0000E94B80DE4CF8091B6018232C1F78C2FEE
:1029E0000E940912811177C0F2CF8091B601823224
:1029F000B1F3C431C9F048F4CB3059F0C031C1F063
:102A00008CE792E00E94BE0511C0C93269F0C8335C
:102A1000B9F782E396E00E94BE0582E892E00E9448
:102A2000BE0581E08170DECF1092BA0280E0FACF5D
:102A30000E94560E8EE792E00E94BE0582E08093CF
:102A4000BA02EFCFC432D0F4CE3108F0C0C0CB30E0
:102A5000E9F048F4C73009F4D1C08BE293E0DF918C
:102A6000CF910C94BE05C331C9F1C431B1F7809147
:102A70002002882349F1109220020AC0CB3409F4C5
:102A8000BBC0C0F4C93299F3C83339F70E94560E5F
:102A900080912002882309F4C8C01F928F9385E299
:102AA00093E09F938F930E9457060F900F900F9083
:102AB0000F9011C0C13509F499C0C23509F490C016
:102AC000CE3459F66AE093C08AE393E00E94BE05D3
:102AD00081E08093BA02DF91CF91089584E193E081
:102AE0000E94BE0582E093E00E94BE05809118011D
:102AF0001F928F938FEF92E09F938F930E945706C0
:102B00008DEF92E00E94BE058BEE92E00E94BE0522
:102B1000809117011F928F9388EE92E09F938F937D
:102B20000E94570686EE92E00E94BE0587ED92E075
:102B30000E94BE05809116011F928F9384ED92E052
:102B40009F938F930E94570682ED92E00E94BE05EC
:102B500081EC92E00E94BE05809115011F928F9337
:102B60008EEB92E09F938F930E9457068CEB92E03E
:102B70000E94BE0587EA92E00E94BE058091140182
:102B80001F928F9384EA92E09F938F930E9457063F
:102B900082EA92E00E94BE058BE892E00E94BE05A8
:102BA000809113011F928F9388E892E09F938F93F7
:102BB0000E94570686E892E00E94BE058DB79EB738
:102BC00048960FB6F8949EBF0FBE8DBF61CFCE5111
:102BD000EC2FF0E0E75DFE4F80818093200258CF1C
:102BE00061E0809120020E94D60C52CF61E080917A
:102BF00020020E94570C4CCF6AE0F3CF8EE1809305
:102C0000180182E3809317018AE08093160184E122
:102C10008093150188E08093140188E2809313016A
:102C20008DE293E00E94BE0533CF82E293E017CF9E
:102C300080E28C0F883068F4C77021E030E001C07A
:102C4000220FCA95EAF78091A002822B8093A002FE
:102C5000A6CE8BE58C0F833070F481E890E0C53A06
:102C600031F083E890E0C63A11F482E890E0DF9119
:102C7000CF910C942A0E88E58C0F873108F069C03B
:102C800082EE90E0C83A09F460C089EE90E0C93A5B
:102C900009F45BC08AEE90E0CA3A09F456C085EBAD
:102CA00090E0CB3A09F451C086EB90E0CC3A09F4BD
:102CB0004CC083EB90E0CD3A09F447C084EB90E040
:102CC000CE3A09F442C087EB90E0CF3AF1F18CECB8
:102CD00090E0C13BD1F18DEC90E0C03BB1F183E8D5
:102CE00091E0C23B91F18AE891E0C33B71F182E946
:102CF00091E0C43B51F184E991E0C53B31F181E2BF
:102D000092E0C63B11F183E292E0C73BF1F084E22E
:102D100092E0C83BD1F085E292E0C93BB1F086E297
:102D200092E0CA3B91F087E292E0CB3B71F08AE2FD
:102D300092E0CC3B51F08FE690E0CD3B31F090E05B
:102D400080E0CE3B11F480E790E0DF91CF910C94CE
:102D5000FE0DCF3B69F40E949D0F9FEF20E782E0BC
:102D6000915020408040E1F700C000000E94250AF9
:102D7000C03F08F4B0CE8C2F0E946B07DF91CF913B
:102D80000C946D0ECF92DF92EF92FF920F931F93F0
:102D9000CF93DF9300D000D01F92CDB7DEB76C0188
:102DA00085E0F601DE01119601900D928A95E1F71A
:102DB000F601408151812381348191E02115310553
:102DC00031F05F3F19F491E04F3F09F090E090FD42
:102DD00099C0F6010281F580F2949FE0F9224983BF
:102DE0005A830B83722F3D832C83602F8D810E9429
:102DF000C608182FE92FE295EF70EF3008F082C077
:102E0000F0E0EB5FF84E0C9453261417141752178A
:102E10005217C817FA178217821710188217E61868
:102E2000E61882178217A219F92FFF70FF2E907FE4
:102E300019F0F29480EFF8220023C9F0FF2039F056
:102E400080919F02F82AF0929F020E943C0F812FEE
:102E50000F900F900F900F900F90DF91CF911F91D7
:102E60000F91FF90EF90DF90CF900C94A914812FD9
:102E70000E94F80FFF2009F445C0F09480919F0252
:102E8000F822F0929F020F900F900F900F900F90EA
:102E9000DF91CF911F910F91FF90EF90DF90CF9036
:102EA0000C943C0F892F8F70907F903211F0829597
:102EB000807F112379F0113009F449C0002309F40F
:102EC00055C0FF2059F0F601958190FF8DC19F708C
:102ED000958304C0002321F1F1100FC00F900F90D3
:102EE0000F900F900F90DF91CF911F910F91FF9056
:102EF000EF90DF90CF900C94EE0F21E0F212EECF26
:102F000080939E020F900F900F900F900F90DF9183
:102F1000CF911F910F91FF90EF90DF90CF90089588
:102F2000F11011C010929E020F900F900F900F9011
:102F30000F90DF91CF911F910F91FF90EF90DF9055
:102F4000CF900C94E30F91E0F912ECCFDBCF00238C
:102F500049F0E5E0EF15B0F29091A002982309F452
:102F6000BDCFE2CFF4E0FF1568F2DECFFF20E1F243
:102F7000812F0F900F900F900F900F90DF91CF91B6
:102F80001F910F91FF90EF90DF90CF900C94F80F6E
:102F9000892F869586958370C1F0813009F0B2CF74
:102FA000812F9370011102C090E080E00F900F908C
:102FB0000F900F900F90DF91CF911F910F91FF9085
:102FC000EF90DF90CF900C94FE0D812F9370011144
:102FD00002C090E080E00F900F900F900F900F9044
:102FE000DF91CF911F910F91FF90EF90DF90CF90E5
:102FF0000C942A0E002389F00E946B070F900F900B
:103000000F900F900F90DF91CF911F910F91FF9034
:10301000EF90DF90CF900C946D0E0E946006EECF83
:10302000892F837009F064C001116CCF812F8295C4
:1030300086958770880F880F412F4F70C42ED12C32
:10304000F12CE12C082E04C0CC0CDD1CEE1CFF1C66
:103050000A94D2F740E050E0BA0114FF11C00FE02B
:1030600010E020E030E004C0000F111F221F331FCA
:103070008A95D2F7B901A801409550956095709551
:103080000091BC021091BD022091BE023091BF029E
:103090009695969593709230E9F028F5913089F0E5
:1030A0004C295D296E297F294023512362237323F4
:1030B0004093BC025093BD026093BE027093BF0266
:1030C00021CFC02AD12AE22AF32A4C295D296E2970
:1030D0007F29EECF4C295D296E297F294027512772
:1030E00062277327E5CF4023512362237323EDCF5B
:1030F0008695002311F0892F8170882309F402CF6F
:10310000812F829586958770880F880F412F4F7089
:10311000C42ED12CF12CE12C082E04C0CC0CDD1CCB
:10312000EE1CFF1C0A94D2F740E050E0BA0114FFF5
:1031300011C00FE010E020E030E004C0000F111FCC
:10314000221F331F8A95D2F7B901A80140955095E7
:103150006095709500915A0210915B0220915C027B
:1031600030915D029695969593709230E9F028F52E
:10317000913089F04C295D296E297F294023512304
:103180006223732340935A0250935B0260935C0264
:1031900070935D02B7CE0C291D292E293F29402BA3
:1031A000512B622B732BEECF4C295D296E297F2981
:1031B0004027512762277327E5CF402351236223FD
:1031C00073234C295D296E297F29DCCF803F09F4C8
:1031D0004EC0D0F480E4810F803270F1002309F4F6
:1031E000ACC0FF2009F4A6C0812F0E94A914193396
:1031F00009F099C0FFEF21EE84E0F15020408040BB
:10320000E1F700C000007ECE823F09F470C008F4F0
:103210005BC0833F19F7002309F47CC0292F2F716D
:1032200081E090E0A0E0B0E004C0880F991FAA1FE1
:10323000BB1F2A95D2F73AC0E12FE071FE2E892FED
:103240008F71002351F00E948C09812F8295807F1D
:10325000F11044CE812F8F7041CE0E946809812FDA
:103260008295807FF11060CE812F8F705DCE00231C
:1032700031F1F4E0FF1508F445CE292F2F7181E0DC
:1032800090E0A0E0B0E004C0880F991FAA1FBB1F08
:103290002A95D2F740915A0250915B0260915C02EC
:1032A00070915D0284279527A627B72780935A023D
:1032B00090935B02A0935C02B0935D0223CE25E065
:1032C0002F1508F41FCED9CF892F8F71002399F0C5
:1032D0000F900F900F900F900F90DF91CF911F9153
:1032E0000F91FF90EF90DF90CF900C948C09892F75
:1032F0008F71002369F30F900F900F900F900F9034
:10330000DF91CF911F910F91FF90EF90DF90CF90C1
:103310000C94680910925A0210925B0210925C029F
:1033200010925D02EFCD133509F464CF173409F024
:10333000E9CD60CF892F8F71CBCFF11019CE892FB6
:103340008F71D9CF8111DECD002309F4DBCD0E942E
:103350009D0F8FEF90E7E2E081509040E040E1F771
:1033600000C000000E94250A1F93CF93DF93809135
:103370002602807FB1F480912302882391F020916E
:10338000580210912702C0912102D0912202A091EF
:103390002402B091250241E0CF3F09F040E0121332
:1033A00004C0DF91CF911F91089581E0109721F023
:1033B000842FDF3F09F080E030E080FD33C0C90199
:1033C00066E070E00E942E26FC01E85DFD4F8181E1
:1033D0008D1328C080818C1325C08281811122C069
:1033E000838194818A1B9B0B883C9105D8F4809142
:1033F00026028F70806180932602C90166E070E02A
:103400000E942E26FC01E35DFD4F90819F7090612C
:10341000908381E292E00E94C216DF91CF911F91CA
:103420000C94AC092F5F3F4F2770B9CF9F92AF929A
:10343000BF92CF92DF92EF92FF920F931F93CF93A1
:10344000DF93CDB7DEB761970FB6F894DEBF0FBE3E
:10345000CDBF8C0185E0F801DE011D9601900D9233
:103460008A95E1F7F80140812181F280C380D48000
:1034700090912102309122026091240270912502E4
:1034800081E06115710531F03F3F19F481E09F3F04
:1034900009F080E0F82FF1709F2E80FD4EC181E28F
:1034A000A82E82E0B82EE0902302F601E61BF70B6F
:1034B000EE2009F404C180912602582F507FE83C89
:1034C000F10508F0BDC0511183C0EF2C321322C0AA
:1034D000941320C0F1101EC08F708061809326026B
:1034E000C5010E94C21680912602F80185838E2DA7
:1034F00061960FB6F894DEBF0FBECDBFDF91CF91BE
:103500001F910F91FF90EF90DF90CF90BF90AF9001
:103510009F90089581E0C114D10431F02F3F19F438
:1035200081E04F3F09F080E080FD14C081E08F25ED
:10353000F82FF170BF2EE09158023091270280FDE4
:1035400022C0FF20A1F28091260281608093260292
:10355000E12CCDCF80E0ECCFF0E0CF0166E070E071
:103560000E942E26DC01A85DBD4F11968C9111970B
:10357000281307C08C91481304C012968C918F11A8
:10358000E0CF3196E770E313E7CF7C2DD98AC88A64
:10359000522F6F2D89890E94C608292F22952F70DE
:1035A000223050F0243078F49F7051F0F80195816A
:1035B000907F31F4E92C9BCF9F7011F08823D1F3D9
:1035C000805E8830B8F3C8010E94C2169B2CF2CFEF
:1035D000321306C0941304C0F801FF2009F48AC016
:1035E0004D872E87FF867C2DD98AC88A522F6F2D52
:1035F00089890E94B609882309F4AEC0FF2009F426
:10360000ABC080912602803270F02091210230916F
:10361000220238872F831986DB86CA868C87CE01E3
:1036200007960E94C21686E0F801A1E2B2E001907E
:103630000D928A95E1F70E94B419EE24E39457CFD6
:1036400051110AC081E292E00E94C21686E0F501A3
:1036500011928A95E9F77CCF32130FC094130DC0F5
:10366000F1100BC0F8018583C8010E94C21686E0E4
:10367000F50111928A95E9F73ACF4D872E87FF869B
:103680007C2DD98AC88A522F6F2D89890E94B6094C
:10369000882309F461C0FF2009F45EC080912602EE
:1036A000803208F220912102309122023A8329834C
:1036B0001B82DD82CC828E83CE010196B2CFE83CA4
:1036C000F105A8F6EF2CFF2009F446C032131FC005
:1036D00094131DC08091260280FD10C0982F907F0A
:1036E00069F0F8018583903F31F0982F907F905FCB
:1036F0008F70892B8583C8010E94C21686E0F8016D
:10370000A1E2B2E001900D928A95E1F7F0CE4D87EB
:103710002E87FF867C2DD98AC88A522F6F2D8989E2
:103720000E94B60981117FCF80912602816080932B
:103730002602C8010E94C216DACEFF2069F04D872A
:103740002E87FF867C2DD98AC88A522F6F2D8989B2
:103750000E94B609811167CFC8010E94C2166DCFC1
:10376000CF93DF93CDB7DEB767970FB6F894DEBF80
:103770000FBECDBF4B8B5C8B6D8B7E8B8F8B1A8A74
:10378000198A85E0FE017396DE011D9601900D9267
:103790008A95E1F786E0FE013D96DE0117960190DD
:1037A0000D928A95E1F7CE0107960E94161A8111B3
:1037B00038C086E0FE013796DE01119601900D9229
:1037C0008A95E1F79F8188852A853B85232B39F0EF
:1037D0008F3F19F481E09F3F19F080E001C081E044
:1037E00080FD1FC08091270290E09C012F5F3F4F1A
:1037F00027703327409158024217130661F166E0A3
:1038000070E00E942E26DC01A85DBD4F96E0FE010F
:10381000319601900D929A95E1F7209327020E942C
:10382000AC098091580290912702891709F190E024
:1038300066E070E00E942E26885D9D4F0E94161A59
:103840008823B1F08091580290E001968770992703
:1038500080935802E6CF0E949D0F1092270210928B
:10386000580286E0E1E2F2E0DF011D928A95E9F775
:1038700067960FB6F894DEBF0FBECDBFDF91CF9134
:10388000089578941F920F920FB60F9211248F9380
:103890009F93AF93BF938091B5029091B602A09190
:1038A000B702B091B8020196A11DB11D8093B50277
:1038B0009093B602A093B702B093B802BF91AF91B4
:1038C0009F918F910F900FBE0F901F9018951F9290
:1038D0000F920FB60F9211248F939F93AF93BF93C4
:1038E0008091A102811113C08091B5029091B6021E
:1038F000A091B702B091B8024196A11DB11D80936D
:10390000B5029093B602A093B702B093B802BF91EC
:10391000AF919F918F910F900FBE0F901F901895B0
:103920001F920F920FB60F9211240F931F932F9394
:103930003F934F935F936F937F938F939F93AF9337
:10394000BF93EF93FF93CF93DF93CDB7DEB7AA97E3
:10395000DEBFCDBF1091E9001F708091EC0080FFA9
:103960003AC080E8182B1092E9008091F000877F20
:103970008093F0007894E4E1F2E08091F10081938B
:1039800082E0EC31F807C9F780911502833009F421
:1039900070C018F5813009F447C0823009F4DAC0EC
:1039A0008091E80083FF15C1809114029091150267
:1039B0009A3008F00EC1E92FF0E0EF51F34E0C946D
:1039C0005326BB1DE11DE91DE11DE91D5C1E7E1E88
:1039D000E91D791F861F80E0C5CF8A3009F4A9C090
:1039E0008B3009F47DC08930D9F680911402813280
:1039F000B9F68091180290911902892B89F680916D
:103A0000E800877F8093E8008091E80082FF2CC067
:103A10008091F1008093EF018091E8008B77809393
:103A2000E8000E94F90ABCCF80911402813A09F0A3
:103A3000B7CF8091E800877F8093E80080911802DB
:103A400090911902892B61F060E090E080E070E0D5
:103A50000E94440A8091E8008B778093E800A0CF11
:103A600060E280EF91E0F3CF809112028111CCCF20
:103A700097CF80911402813A09F092CF8091180279
:103A800090911902892BA1F48091E800877F80939F
:103A9000E8008091E80080FFFCCF809112018093C4
:103AA000F1008091E8008E778093E8000E94F90A87
:103AB0008091180290911902019709F071CF8091BD
:103AC000E800877F8093E8008091E80080FFFCCFCA
:103AD000809110018093F1008091E8008E779FCF54
:103AE00080911402813209F05BCF8091180290918D
:103AF0001902892B59F48091E800877F8093E800B0
:103B00000E94F90A80911602809312018091180296
:103B100090911902019709F043CF8091E800877FC7
:103B20008093E8000E94F90A8091160280931001A8
:103B300037CF80911402813209F032CF8091E800B2
:103B4000877F8093E8000E94F90A80911702809392
:103B5000B90226CF80911402813A09F021CF8091D9
:103B6000E800877F8093E8008091E80080FFFCCF29
:103B70008091B902AFCF803889F0823851F58091B9
:103B800018028F70853028F58093E9008091EB0052
:103B900085FB882780F91092E90006C08091100209
:103BA00090911102911182609091E800977F90931B
:103BB000E8008093F1001092F1008091E8008E7788
:103BC00049C0282F2D7F29F48823B1F1823009F4D0
:103BD00046C08091E80083FF0AC08091E800877F9B
:103BE0008093E8008091EB0080628093EB0010925C
:103BF000E9008091F00088608093F0001F701093BE
:103C0000E900AA960FB6F894DEBF0FBECDBFDF91D4
:103C1000CF91FF91EF91BF91AF919F918F917F9144
:103C20006F915F914F913F912F911F910F910F9045
:103C30000FBE0F901F90189580911602813049F6A3
:103C4000933009F080E0809311021092E900809196
:103C5000E800877F8093E8000E94F90ABACF80913C
:103C600016028111F2CF809118028F702FEF280F6A
:103C7000243008F0AECF8093E9002091EB0020FFC4
:103C8000E4CF933031F48091EB0080628093EB00BD
:103C9000DCCF9091EB0090619093EB0021E030E05D
:103CA00001C0220F8A95EAF72093EA001092EA00F9
:103CB0008091EB008860EACF81118BCF00911602D2
:103CC0000F778091E3008078802B8093E3008091D0
:103CD000E800877F8093E8000E94F90A8091E8005D
:103CE00080FFFCCF8091E30080688093E30083E055
:103CF000011101C082E0809312026BCF80588230A4
:103D000008F067CF20911602309117022C3DA3E0F6
:103D10003A07A1F583E08A838AE289834FB7F89452
:103D2000DE01139620E03EE051E2E32FF0E05093F5
:103D30005700E49120FF03C0E295EF703F5FEF7002
:103D40008E2F90E0EA30C0F0C7968D939D932F5F41
:103D5000243159F74FBF8091E800877F8093E800B6
:103D60006AE270E0CE0101960E94440A8091E80068
:103D70008B778093E8002DCFC096E7CF8091180213
:103D800090911902432F55274330510509F44FC034
:103D900078F54130510509F445C084E590E0EAED3D
:103DA000F1E04230510509F014CF2091E800277F5F
:103DB0002093E80020911A0230911B02821793078A
:103DC00008F49C0140E02115310509F063C0411160
:103DD00061C08091E80082FDC9CF809112028823E2
:103DE00029F2853019F28091E80083FFF2CFBECF2F
:103DF0004132510509F43FC04232510509F0E9CE84
:103E00008330910508F0E5CEFC01EE0FFF1FE35E65
:103E1000FE4F0190F081E02D865E9E4FDC018C917B
:103E200090E01DC082E190E0EEE2F2E0BECF3327E9
:103E300021303105C1F060F02230310509F0C9CEE2
:103E4000E0E4F2E0E4918E2F90E0E0E4F2E007C0DD
:103E5000EAE5F2E0E4918E2F90E0EAE5F2E00097E7
:103E600009F4B7CEA2CFE0E5F2E0E4918E2F90E026
:103E7000E0E5F2E0F4CF8330910508F0AACE880F98
:103E8000991FFC01ED5DFE4F0190F081E02D89E06E
:103E900090E08BCF80911202882309F467CF8530A0
:103EA00009F464CF8091E80083FD60CF8091E80041
:103EB00082FD8FCF8091E80080FF85CF8091F20056
:103EC00090E02115310519F08830910550F041E05E
:103ED000089709F040E08091E8008E778093E80031
:103EE00072CF44914093F1003196215031090196EF
:103EF000E8CF803809F06DCE8091E800877F80930D
:103F0000E800809113028093F10057CE811161CEB9
:103F100000911602023008F05CCE8091E800877FA5
:103F20008093E800009313020E94F90A002399F09D
:103F300084E08093120242E261EC81E00E94180B5F
:103F400042E061EC82E00E94180B46E261EC83E003
:103F50000E94180B3ECE8091E30087FDE9CF81E0FF
:103F6000E8CF1F920F920FB60F9211242F933F9319
:103F70004F935F936F937F938F939F93AF93BF9371
:103F8000EF93FF938091E10082FF09C08091E200EE
:103F900082FF05C08091E1008B7F8093E1008091DA
:103FA000E10080FF1FC08091E20080FF1BC0809174
:103FB000E2008E7F8093E2008091E2008061809336
:103FC000E2008091D80080628093D80019BC85E01F
:103FD000809312028091EF018093EE011092EF0125
:103FE0000E949D0F8091E10084FF2DC08091E2002E
:103FF00084FF29C084E089BD86E089BD09B400FE44
:10400000FDCF8091D8008F7D8093D8008091E10012
:104010008F7E8093E1008091E2008F7E8093E200AA
:104020008091E20081608093E200809113028823F6
:1040300009F45DC084E0809312020E949D0F80917C
:10404000EE018093EF018091E10083FF3FC08091FA
:10405000E20083FF3BC08091E100877F8093E10015
:1040600082E080931202109213028091E1008E7F11
:104070008093E1008091E2008E7F8093E200809146
:10408000E20080618093E20042E060E080E00E9414
:10409000180B8091F00088608093F00081E080939D
:1040A00012011092B9021092EF0180E2E0EFF1E00C
:1040B000DF011D928A95E9F7E7EBF1E01192B1E09B
:1040C000E63DFB07D9F781E080931001FF91EF9166
:1040D000BF91AF919F918F917F916F915F914F9120
:1040E0003F912F910F900FBE0F901F9018958091C8
:1040F000E30087FD02C081E09ECF83E09CCFCF9399
:10410000DF93CDB7DEB72C970FB6F894DEBF0FBEA6
:10411000CDBF84B7877F84BF0FB6F894A8958091F0
:104120006000886180936000109260000FBE80E89C
:1041300090E00FB6F89480936100909361000FBEF9
:1041400085E69BE0909335018093340186E091E011
:104150009093AD028093AC0281EC91E00E94BE0589
:104160000E940E0A809163008E7F8093630081E03D
:104170008093ED011092E2001092E1008091D8004E
:104180008F778093D8008091D80080688093D80082
:104190008091D8008F7D8093D80084E089BD86E02F
:1041A00089BD09B400FEFDCF1092120210921302D5
:1041B000109211021092100242E060E080E00E9432
:1041C000180B8091E1008E7F8093E1008091E200E6
:1041D00081608093E2008091E20088608093E20039
:1041E0008091E0008E7F8093E000789482E084BD2F
:1041F00093E095BD9AEF97BD80936E000E944E0CA0
:1042000084B114B885B18FEF85B9EAEDF1E08AEA9F
:1042100092E022EA32E03C872B87AB85BC851D9279
:10422000BC87AB8711928A179B07B9F78091BB02B5
:104230008D7F8093BB023D9A459ABFEFE9E6F8E196
:10424000B150E040F040E1F700C000003D984598D3
:1042500090E080E00E94CC248D3E9E4FD1F06DEE28
:104260007EEF90E080E00E94E02460E082E090E059
:104270000E94D22460E083E090E00E94D22460E0BB
:1042800084E090E00E94D22460E085E090E00E940B
:10429000D22489E691E00E94BE0515E61150B9F5D9
:1042A00082E691E00E94BE0589E290E00E943F080C
:1042B000811111C18AE290E00E943F088823F9F041
:1042C0006FEF7FEF90E080E00E94E0246FEF82E0EC
:1042D00090E00E94D2246FEF83E090E00E94D2240D
:1042E0006FEF84E090E00E94D2246FEF85E090E0D1
:1042F0000E94D2246FEF86E090E00E94D22485E0F5
:1043000090E00E943F08882359F00E94250A0E94ED
:1043100056118FE39CE90197F1F700C00000BECF72
:1043200090E080E00E94CC248D3E9E4F09F0C7C0F3
:1043300082E090E00E94C4248093BB0287E090E07A
:104340000E943F08882379F08BE190E00E943F08AB
:10435000882309F4F2C19091BB02892F8D7F91FFD0
:1043600082608093BB026091BB0282E090E00E9479
:10437000D22484E090E00E94C424F82E80EE90E0E5
:104380000E943F08882321F0F094F0FAF094F0F8AE
:1043900089E390E00E943F08882321F0F094F1FA2D
:1043A000F094F1F882EE90E00E943F08882321F01B
:1043B000F094F2FAF094F2F886EE90E00E943F0852
:1043C000882321F0F094F3FAF094F3F883EE90E070
:1043D0000E943F08882321F0F094F4FAF094F4F856
:1043E00085E390E00E943F08882321F0F094F5FADD
:1043F000F094F5F881E390E00E943F08882321F0D3
:10440000F094F6FAF094F6F881E190E00E943F080B
:10441000882321F0F094F7FAF094F7F86F2D84E0F8
:1044200090E00E94D224F7FE06C08091110191E035
:1044300089278093110187E290E00E943F08182F9E
:104440008EE190E00E943F08811112608FE190E0C0
:104450000E943F088111146080E290E00E943F08B2
:104460008111186081E290E00E943F088111106183
:1044700082E290E00E943F088111106283E290E0A6
:104480000E943F088111106484E290E00E943F087E
:10449000882309F471C11068612F83E090E00E94C5
:1044A000D224812F90E0B0E0A0E08093BC029093F2
:1044B000BD02A093BE02B093BF02F09259020E94C7
:1044C0005611E2EAF2E081918111F9CF2B853C850A
:1044D0002E173F07C1F7809112028430E1F70E9446
:1044E0004D0B8823C1F38FEA91E00E94BE0581EA5B
:1044F00091E00E94BE05A6E94A2EA1E05A2EB8E13D
:104500006B2E712C80911202853009F43CC10E94FF
:104510005611E3EEEE2EE1E0FE2EF2EAAF2EF2E0CF
:10452000BF2E312CD5012D905D01F70190809214A2
:1045300009F464C08091BB0281FF3CC089E891E02E
:104540000E94BE0502EA12E0D12CC12CD8012D91A7
:104550008D01229530E0C901880F991F880F991F9E
:104560008C7C35952795359527952373822B90E084
:10457000E9E1F1E0FF93EF939C01220F331F2A7AC8
:10458000959587958575822B1F928F93DF92CF9299
:104590008EE791E09F938F930E945706BFEFCB1A4F
:1045A000DB0A0FB6F894DEBF0FBECDBFF8E0CF1622
:1045B000D10461F6C12CDD24D3949224892D8D2160
:1045C000C1F0CE823F8291E0822D8D2109F490E0EE
:1045D00098870E9451088160782F9A8789874E8139
:1045E0005F8168858A850E94B01BD7018C918D25DB
:1045F0008C93C394DD0CB8E0CB12E0CF3394EFEF93
:10460000EE1AFE0AF8E03F128DCF2FEF29832A839E
:104610001B820E9451088160782F9D838C83498181
:104620005A816B818D810E94B01B8091AE02909166
:10463000AF022FB7F8944091B5025091B602609145
:10464000B7027091B8022FBFFA01E81BF90B209155
:10465000AB028091170190E0211107C080911801F1
:1046600090E06AE070E00E942E26E817F90780F0DB
:104670008091B102D090B202F090B302E090B40207
:104680008111B9C0D1107CC1F1107AC1E11078C19B
:104690000E94020A9091E2018917C9F00E94020A61
:1046A0008093E2019091BB029570953051F41F9276
:1046B0008F935F924F920E9457060F900F900F902A
:1046C0000F908091E20181FF04C13D9A459A2091AB
:1046D000E4003091E5008091EB019091EC01281706
:1046E000390709F40FCF8091E4009091E500909391
:1046F000EC018093EB010E944D0B882309F402CF5B
:1047000080911202843009F0FDCE8091E9008F7013
:104710009091EC0090FFE0C090E8892B93E090939B
:10472000E9009091EB0090FF04C09091EE0097FD9E
:10473000F1C08F708093E900E5CE8EE090E00E949A
:104740003F08882339F09091BB02892F8B7F92FF1D
:10475000846007CE80E190E00E943F089091BB0208
:10476000882329F0892F877F93FF8860FACD892FCE
:104770008E7F90FF8160F5CD11118ECE83E090E0A9
:104780000E94C4248FCE80911202843011F11092C5
:10479000A10280E40FB6F894A895609260000FBE65
:1047A0008093600083B7817F846083BF83B781601B
:1047B00083BF7894889583B78E7F83BF0FB6F894B4
:1047C000A8958091600088618093600010926000DD
:1047D0000FBE80911102882309F494CE0E945611D5
:1047E000E2EAF2E081918111B5C08B859C858E173C
:1047F0009F07C1F787CE2F3F19F02F5F2093AB02A1
:10480000181624F40E941F078093B1028091B10210
:1048100087FF05C00E941F0781958093B1021D1478
:1048200024F40E941F078093B2028091B20287FF96
:1048300005C00E941F0781958093B2026091B1026A
:10484000662331F1D090B202DD2011F1062E000C6A
:10485000770B880B990B0E942D2523E333E343E369
:104860005FE30E9491250E94F5246093B1026D2DB3
:10487000DD0C770B880B990B0E942D2523E333E386
:1048800043E35FE30E9491250E94F5246093B20206
:104890001F1424F40E94E4068093B3028091B302B3
:1048A00087FF05C00E94E40681958093B3021E1421
:1048B00024F40E94E4068093B4028091B40287FF3E
:1048C00005C00E94E40681958093B4020E946D0E9B
:1048D000DFCE3D984598FBCE90E01FCFE0910101DF
:1048E000F0910201E90FF11D20819F5F30910501D8
:1048F0009323909304012093F1009091E80095FD9B
:1049000009C09091E80090FF05C09091E8009E7763
:104910009093E8009091040120910301291721F060
:104920002091E80025FDDACF9091F200992309F457
:1049300000CF9091E80090FFFCCE9091E80095FDAB
:1049400006C09091E8009E779093E800F2CE109216
:10495000F100F3CF84E089BD86E089BD09B400FE93
:10496000FDCF8091D8008F7D8093D8008091E000AA
:1049700082608093E0008091E00081FDFCCFC2CD99
:104980002F3F09F03ACF4BCFF999FECF92BD81BDB1
:10499000F89A992780B50895A8E1B0E042E050E088
:1049A0000C94E724262FF999FECF1FBA92BD81BD42
:1049B00020BD0FB6F894FA9AF99A0FBE01960895A1
:1049C0000E94D224272F0C94D324DC01CB01FC01BC
:1049D000F999FECF06C0F2BDE1BDF89A319600B458
:1049E0000D9241505040B8F708950E94FC246894FD
:1049F000B1110C948B2508950E94702588F09F5763
:104A000098F0B92F9927B751B0F0E1F0660F771FF2
:104A1000881F991F1AF0BA95C9F714C0B13091F0E8
:104A20000E948A25B1E008950C948A25672F782F7B
:104A30008827B85F39F0B93FCCF3869577956795AD
:104A4000B395D9F73EF490958095709561957F4F19
:104A50008F4F9F4F0895E89409C097FB3EF49095BF
:104A60008095709561957F4F8F4F9F4F9923A9F047
:104A7000F92F96E9BB279395F695879577956795D6
:104A8000B795F111F8CFFAF4BB0F11F460FF1BC01A
:104A90006F5F7F4F8F4F9F4F16C0882311F096E9AD
:104AA00011C0772321F09EE8872F762F05C066235B
:104AB00071F096E8862F70E060E02AF09A95660F14
:104AC000771F881FDAF7880F9695879597F90895CD
:104AD00057FD9058440F551F59F05F3F71F04795AF
:104AE000880F97FB991F61F09F3F79F08795089594
:104AF000121613061406551FF2CF4695F1DF08C0B3
:104B0000161617061806991FF1CF869571056105CF
:104B100008940895E894BB2766277727CB0197F977
:104B200008950E94A3250C941D260E940F2638F09C
:104B30000E94162620F0952311F00C9406260C9462
:104B40000C260C948B250E94682578F39923C9F3D1
:104B50005523B9F3950F50E0551FAA27EE27FF27DD
:104B6000BB2700240894679520F4E20FF31FB41FBD
:104B70000A1E220F331F441FAA1F6695A9F77795B7
:104B800030F4F30FB41F0A1E121E08F46395330F9E
:104B9000441FAA1F221F769599F7879520F4B40F1A
:104BA0000A1E121E631F440FAA1F221F331F869561
:104BB000A9F7862F712D602D11249F5750409AF030
:104BC000F1F088234AF0EE0FFF1FBB1F661F771F0F
:104BD000881F91505040A9F79E3F510580F00C94DA
:104BE00006260C948B255F3FE4F3983ED4F386951C
:104BF00077956795B795F795E7959F5FC1F7FE2B7A
:104C0000880F911D9695879597F9089597F99F6755
:104C100080E870E060E008959FEF80EC0895002444
:104C20000A941616170618060906089500240A9411
:104C300012161306140605060895092E0394000C97
:104C400011F4882352F0BB0F40F4BF2B11F460FF26
:104C500004C06F5F7F4F8F4F9F4F089500245527EB
:104C600004C0080E591F880F991F009729F07695E8
:104C70006795B8F37105B9F7802D952F089597FBC7
:104C8000072E16F4009407D077FD09D00E9459260C
:104C900007FC05D03EF4909581959F4F089570953F
:104CA00061957F4F0895EE0FFF1F0590F491E02D61
:104CB0000994AA1BBB1B51E107C0AA1FBB1FA61763
:104CC000B70710F0A61BB70B881F991F5A95A9F7B5
:0E4CD00080959095BC01CD010895F894FFCF1A
:104CDE0005360100007F4A0B0311D51095105D10AB
:104CEE000101012808140A321E00397F221501968F
:104CFE00007400EC0105021E020102030405060702
:044D0E000809000090
:106800000000000000000000040005000600070072
:10681000080009000A000B000C000D000E000F001C
:1068200010001100120013001400150016001700CC
:10683000180019001A001B001C001D001E001F007C
:10684000200021002200230024002500260027002C
:10685000280029002A002B002C002D002E002F00DC
:1068600030003100000033003400350036003700BE
:1068700038003900000000000000000000000000A7
:106880000000000000000000000000000000000008
:1068900000000000000000000000000000000000F8
:1068A00000000000000000000000000000000000E8
:1068B00000000000000000000000000000000000D8
:1068C00000000000000000006400E700000000007D
:1068D00000000000000000000000000000000000B8
:1068E0000000000000000000320000000000000076
:1068F000E000E100E300E200E400E500E6006500FE
:00000001FF
